:101B7B004856522D31363030000134000000436F8F
:101B8B006E74726F6C000100400418000001556404
:101B9B00656D616E64000100410418000001556D14
:101BAB006561730000000100450406FA0001496DF0
:101BBB00656173000000010049013400000053749B
:101BCB0061747573000001004D015C0000005472DC
:101BDB006970436E740001004E04180000015261DD
:101BEB006D705570000001004F0418000001526128
:101BFB006D70446F776E0100530418000001556C33
:101C0B00696D697400000100570406FA0001496C04
:101C1B00696D6974000001005B0406FA000152490A
:101C2B006C696D69740001005F015C000000547207
:101C3B0069704D617800010063010300000054726C
:101C4B00697054696D65010064045D0000094144CD
:101C5B00436761696E000100650418000009414487
:101C6B00436F66730000010069045D000009444185
:101C7B00436761696E0001006D041800000944415F
:101C8B00436F66730000010071045D00000943554A
:101C9B0052766761696E010075045D00000943555A
:101CAB00526761696E000100790406FA0009435519
:101CBB00526F6673000001007D0418000009554443
:101CCB004143000000000100810000000000000003
:091CDB0000000000000000000000
:0B30BB000175100309FF1B84010800D1
:100F870075F045E53C900041120E26120D9FE53C99
:100F970025E025E024E0F582E43404F583120DD042
:100FA700E53C25E025E024E0F582E43404F58312EE
:100FB7000D9FE53C90008175F045020E26F075F017
:100FC70045E53C90004D120E26E054FBF0E53C75DC
:100FD700F04590004D020E2675F045E53B90004127
:100FE700120E26120D9F78BFE4FBFAF912080F9034
:100FF7000081E53B75F045020E26E53C25E025E03E
:1010070024E0F582E43404F583120D9FE53C90005B
:101017004175F045020E26E53E75F04590005B02EE
:101027000E2675F045E53B900045120E26120DB8C9
:10103700900041E53B75F045020E26E054BFF07481
:1010470090253CF582E43404F5832275F045E53CB0
:1010570090005F120E26120D9FE53C90004975F037
:1010670045020E26C3740F953C25E025E024ADF517
:1010770082E43406F583120D9F7801120D46C8EC01
:10108700C8C9EDC9CAEECACBEFCB7E00E53E540115
:10109700FFE4FCFD120D04C3740F953C25E025E029
:1010A70024ADF582E43406F58322E53E75F04590DC
:1010B7000057020E26120D9FE53C25E025E024E0AF
:1010C700F582E43404F5832290004F75F045020E53
:1010D7002690005375F045020E2675F045900040A6
:1010E700020E2675F04590004E020E2675F04590CB
:1010F7000064020E26E53B25E025E024A0F582E406
:101107003404F5832275F045900079020E2675F0B8
:1011170045E53C120E26120DB812090079C878422F
:10112700E4FBFA020A09CBEFCBE53C25E025E024F6
:1011370000F582E43400F58322120D9FE4FBFA22C6
:10114700120DB8020AA675F045E53B020E261208F5
:101157000B9006A9120DD09006A9020D9FE5102449
:1011670003F8120DAB020AA6797A7844E4FBFA0277
:101177000A09120D9F7B007A3C791C7846020AA661
:101187005420FCE4FBFAF9F8C3020D357B00120981
:1011970000E4FBFAF9783F2275F045E53E020E269A
:1011A700E7A8100808F6A810E4F6A8100822AB3B39
:1011B700AA3CA93D020BD2C8ECC8C9EDC9CAEECA00
:1011C700CBEFCB22120A09E4FBFA792078402212EE
:1011D7000DD0E53DC313F53DE53E13F53E053CE572
:1011E7003C22120D9FE51024FCF510F822E5475428
:1011F700C0FFE546FEE545FDE544541FFC22900689
:10120700A9120DB8020900C2CD08C9E8C9A810087B
:1012170008E65794002275F045E53B020E26900636
:10122700A9120DD0E4FFFE227B007A247974784955
:10123700221510A810EFF615101510228F4B8E4AA5
:0A1247008D4922AB41AA42A94322BF
:1016DF0075840F75A4FD75A5FF75A6FF75A7FF751A
:1016EF009CFEE4F59DF59E759FFFD2B4EF7003024B
:1016FF0017877E047F507D007B017A007940120EA0
:10170F00AAE4F53E1210B1120DF542480000121076
:10171F001E120DF54348000090005F12119F120D2D
:10172F00F543480000E53E1210CF120DF5412000A1
:10173F0000E53E1210D8120DF541200000E53E12D3
:10174F0010F3740AF090006512119F120DF53F808F
:10175F00000075F045E53E90006D120E26120DF556
:10176F003F800000E53E12110C120DF53F80000086
:10177F00053EE53E6410708CE4F53EE53E1210E147
:10178F007402F0E53E120FD6E4F0E53E121015128A
:10179F000DF500000000E53E1210EAE4F01210B162
:1017AF0012114079487842120AA6500A1210B1124B
:1017BF000DF54248000012101E121140794878436F
:1017CF00120AA6501212101E121179600A12101E60
:1017DF00120DF543480000E53E1210C1120DF50041
:1017EF000000001230FBE53E121132120DD0053E03
:1017FF00E53EC3941040847861B6FF0A08B6FF0631
:10180F00187603087620E4F53E75F045E53E900026
:10181F004D20B409120E26E04401F08007120E2667
:10182F00E054FEF0053EE53EB410DE75840FD2CED7
:10183F00D2A17F017E00122CF5C2A07F017E001283
:10184F002CF5C2A175D8FF75E8FFE4F53E7490251D
:10185F003E12104A7409F0053EE53EB410EFE4F570
:10186F003E7D01AF3E12000E053EE53EC394104093
:10187F00F0E4F53EE53E1210FE120DF500000000FB
:07188F00053EE53EB410ED3B
:01189600222F
:10284C001510A810EFF6A810E6FF600864016004EC
:10285C00EFB404171228E8120FD9E054DFF012314C
:10286C001A74902F12104AE04401F0A810E6640884
:10287C00702D12311AEF1210B312114079487842B0
:10288C00120AA6500D1228E81210B6120DF5424885
:10289C00000012311A74902F12104AE04401F0A873
:1028AC0010E66409703312311AEF12102012114025
:1028BC0079487843120AA6502012311A75F045EF68
:1028CC00121023121179601112311A75F045EF12A2
:1028DC001023120DF54348000005102212311A7511
:0428EC00F045EF22A2
:050003008F347F002294
:093111008B348A3589367F0022D7
:101FA60015101510A810ECF608EDF61212381510DB
:101FB60075840FE5102403F8E6C394085004C2CCD8
:101FC6008002C2CB1220D41211AD7608A810E6C347
:101FD60094045023C2CD08E6540394004003D380F2
:101FE60001C31220A3A81008E8C0E0E6C313FFD07F
:101FF600E01220C90680D51211AD7608A810E6C3F6
:102006009404502CC2CDE5102403F8E65407A8101A
:102016000856D394004003D38001C31220A3A8100E
:1020260008E8C0E0E6C313FFD0E01220C90680CC62
:10203600E5102404F91211A77680A810E6C39408C7
:10204600501D12120E4003D38001C31220B6A810F1
:1020560008E8C0E0E6C313FFD0E01220E180DBE52C
:10206600102404F9091211A77680A810E6C3940873
:10207600501D12120E4003D38001C31220B6A810C1
:1020860008E8C0E0E6C313FFD0E01220E180DBD20F
:06209600CCD2CB1220D4D5
:10209C00E5102406F5102292CA7F017E00122CF561
:1020AC00D2CD7F017E00122CF52292CA7F017E00D8
:1020BC00122CF5D2CD7F017E00122CF522F8EFF612
:1020CC007F01123079A810227F017E00122CF57F3F
:1020DC000112307922F8EFF67F01123079A8100640
:0120EC0022D1
:061CE4008B3E8A3F89409F
:101CEA0075840F121E36C2C9121E40A2C8E433F50B
:101CFA0047754600754500754400E4FFFEFDFCABE0
:101D0A0047AA46A945A844D3120D354008D2C9129C
:101D1A001E407F0022AB3EAA3FA940E508120C18DC
:101D2A00E50804540FF508E4F54BF54AF5497548FA
:101D3A00B0E50830E012E54BFFE54AFEE549FDE56E
:101D4A00484408121243F548E508C313FFE4FCFDB2
:101D5A00FE7818120D46E54B4FFFE54A4EFEE5495F
:101D6A004DFDE5484C121243F548E4F547F546F5B2
:101D7A0045F544F54CAF47AE46AD45AC4478011243
:101D8A000D468F478E468D458C44A2C8E43345479D
:101D9A00FFE546FEE545FDE5448F478E468D45F550
:101DAA0044E4FFFEFDE54854801211895002800187
:101DBA00C392CAAF4BAE4AAD49AC487801120D4640
:101DCA001212438C48D2CD7F017E00122CF5121ECE
:101DDA0036054CE54CC39420409BD2C9C2CDE4FFE2
:101DEA00FEFDE54412118770091211F4EC44E0FC7F
:101DFA0080041211F4E4120B13E4FBFAF9784E1280
:101E0A0011CB12090012124A120D7912124A120D3E
:101E1A005912123112119312080F12279C12122F03
:0B1E2A00120A0912124A120D797F0102
:101E350022C2CD7F017E00122CF5227F017E001289
:031E45002CF52257
:0320ED0012123894
:1020F000A8100808E6900057120FBE12114079A0F0
:10210000784012080F121164A810602440220808B9
:10211000E6FB900057120FFB120D9FE5102403F809
:10212000120DC475F045EB120FD9E04410F0800A8F
:102130000808E6120FD6E054EFF0E4FFFEFD7C3F06
:10214000121164600D400B7D00A8100808E6FF1214
:10215000000EA8100808E690006D121018120D9FCE
:10216000E5102403F8120DAB120900A8100808E6C8
:1021700090007112103C120DB812080FE5102403E4
:10218000F8120DC4E4FFFEFDFC121164500CE510C2
:102190002403F8120DDC00000000E5102403F8E829
:1021A000C0E0120D9379A87841121127D0E0F812FF
:1021B0000DC4E4FFFE7D207C40121164600E400CD3
:1021C000E5102403F8120DDC402000001211CEE8C7
:1021D000C0E0E5102403F8120D93D0E0F8120A09CC
:1021E0007AFF797F784712119312080F120B51A8CA
:1021F00010EEF608EFF6A810E6FC08E6FDA81008B9
:0622000008E6FF121FA614
:07220600E5102407F510228A
:062988008B3B8A3C893DF7
:10298E007541017542067543A9121CE4EF7002FFF2
:10299E00229006A9121140792E7842120900900653
:1029AE00A9120DD01211B5900065121065120D9F6F
:1029BE001212051211B59000691210D2120DB81232
:1029CE00080F1212257D7A7C4412120512279C12D2
:1029DE00116F121225FD7C3F9006A912114760055A
:1029EE004003D38001C340047D0180027D0012119B
:1029FE00B5FF12000EC2AF9006A9120D9F1211B5AF
:0D2A0E009000451210DB120DD0D2AF7F01F9
:012A1B002298
:101E4800E4F53B75F045E53B121023120D9FE53B89
:101E580012106212114760025003021EFE75F0450F
:101E6800E53B1210231211797003021EFE1210FCBA
:101E780012114012118D70091230FB1210FC120D54
:101E8800D01211EC120DDC00000000AF3B1220ED67
:101E9800E53B1210C1120DF500000000E53B120FE2
:101EA800BB120DF5000000007490253B12104AE0AB
:101EB80054FEF07490253B12104AE054FDF07490E3
:101EC800253B12104AE054FBF075F045E53B120F34
:101ED800D9E054F3F075F045E53B120FD9E0FF2047
:101EE800E51475F045E53B120FD9EF4420F0E53BCA
:101EF8001210EAE004F075F045E53B120FD9E03026
:101F0800E57875F045E53B900063120E26E0FF7515
:101F1800F045E53B1210EDE0C39F505E1230FBEC3C
:101F2800C0E0EDC0E0EEC0E0EFC0E0E53B1210F32A
:101F3800E075F064A4FFAEF0E4FCFD1210FC120D95
:101F4800B8120CF71211BED0E0FFD0E0FED0E0FDD1
:101F5800D0E0FCD3120D35502175F045E53B120F4A
:101F6800D9E054DFF01210FC120DF50000000074E7
:101F780090253B12104AE04401F075F045E53B120C
:101F88000FD9E030E50B7A007B647D03AF3B122E5E
:0D1F98003D053BE53BC394105003021E4B7A
:011FA5002219
:101A0E0075840FC2A1121B73AFD8EFADE8F53DED93
:101A1E00F53ED39400E53D94004009D2A17F017EAE
:101A2E0000022CF5E4F53BE53B1210A3120DF50078
:101A3E00000000053BE53BB410EDE4F53BAFD87577
:101A4E003D008F3EE4F53C12106B1211D6B408F730
:101A5E00AFE8753D008F3E753C0812106B1211D623
:101A6E00B410F7D2A0121B73C2A07F017E00122CFD
:101A7E00F5053BE53BC3942040C3D2A1C2A0E4F5DB
:101A8E003BE53B1210A3120D9FE4FFFEFDEC12117D
:101A9E00877012E53B1210A3120D9FEC541FFCEC45
:101AAE0044E0FC800DE53B1210A3120D9FEC541F79
:101ABE00FCE4120B137980784D1211731211CE12B1
:101ACE0009009006A9120DD07B1F7A85790F7841F7
:101ADE0012115E120A0912116F12122F1209001240
:101AEE001158ECC0E0EDC0E0EEC0E0EFC0E09000B9
:101AFE004512114D120D9F90007512114D121208C4
:101B0E001211BED0E0FFD0E0FED0E0FDD0E0FC121E
:101B1E00115590007D12121D120DB8121155E53B94
:101B2E0012110C1212089006A91212287D7A7C440A
:101B3E009006A9120DB812119512080F12279C12B9
:101B4E00116F9006A9120DD0C2AF12115E9000490E
:101B5E0012121D120DD0D2AF053BE53BC3941050AF
:041B6E0003021A8FC5
:091B7200227F017E00122CF522F5
:1014F200E4F53CE53C1210E1E020E0030216A812FC
:101502000FD4E030E5030216A8121046E030E07472
:101512001210011211476030402EE53C1210CF121A
:101522001140F9F8120AA6501F121046E0440212A6
:101532001045120FD0E04404120FD3E054F7120FFB
:10154200D3121042E054FEF0121001121147502B38
:10155200E53C1210D8121140F9F8120AA6501C12DA
:101562001046E054FD121045E04404120FC4E0445A
:1015720008120FD3121042E054FEF01230FB121187
:1015820030120DD0121046E020E10302162D123067
:10159200FB12112D120D9FC3EB9FF53B121052123D
:1015A200114775F045600D400BE53C120FD9E04440
:1015B20040F08009E53C120FD9E054BFF0E53B60F2
:1015C2006A12105212114750621210BFC083C082B9
:1015D200120DB8E8C0E0E9C0E0EAC0E0EBC0E0AC60
:1015E2003BE4120B1D90004F121115D0E0FBD0E02E
:1015F200FAD0E0F9D0E0F812080FD082D083120FAF
:10160200A4120DD01210131210BC12114740131263
:101612000F87120DD0121046E054FD120FC4E05491
:10162200BFF01210BF1216BA120DD0121046E030DF
:10163200E2741230FB12112D120D9FC3EB9FF53B8A
:1016420060641210BFC083C082120D9FECC0E0ED37
:10165200C0E0EEC0E0EFC0E0AC3BE4120B1D900036
:10166200531211151211BED0E0FFD0E0FED0E0FD02
:10167200D0E0FC12080BD082D083120FA4120DD03E
:101682001210131210BC12114760025010120F8771
:10169200120DD0121046120FD0E054F7F01210BF04
:1016A2001216BA120DD07F00123079053CE53CC308
:0716B200941050030214F52F
:1016B90022120D9FE51024FCF510F8120DC4AF3C61
:1016C9001220ED1230FBE53C25E025E02400F582EF
:0616D900E43400F5832259
:101897008F3B75F045EF1210E4E0FF20E0030219DB
:1018A700C07490253B12104AE0540660030219C029
:1018B70075F045E53B120FD9E030E5030219C0EF9B
:1018C70020E103021988900041120FF9120D9FE5DC
:1018D7003B1210C1120DD0121029120D9F12080BC6
:1018E7001230D7E4FBFA79A878411211CB120A0912
:1018F700E4FBFA79807847121195120AA640030291
:1019070019C0120FF6C083C082120DB8E8C0E0E913
:10191700C0E0EAC0E0EBC0E0121029120D9F1208E8
:101927000BD0E0FBD0E0FAD0E0F9D0E0F812080FD6
:10193700D082D083120DD0120FDF1211475006123A
:101947000FDF120DD0121037120D9F783F120FEFD5
:101957001211476011400F121037121140F9783FEA
:10196700120FF3120DD07490253B12104AE054FE6B
:10197700F0120FF61211E9120DC4AF3B1220ED80E1
:10198700387490253B12104AE030E02D12103712C0
:101997000D9FE53B1210C1120DD0121037120D9F8B
:1019A700120FF6120DD01210371211E9120DC412D0
:1019B7001A0412104AE054FEF090004012103AE068
:1019C70020E0357490253B12104AE030E02A120FD0
:1019D700F6120DF500000000E53B1210C1120DF5DF
:1019E700000000001211EC120DDC00000000121ABA
:1019F7000412104AE054FEF07F01023079AF3B1227
:071A070020ED7490253B2245
:102F9D007F00123079121A0E1230FBE47B2C7A016D
:102FAD0012118D5017121E481214F27B007A0079FF
:0C2FBD003A122988EF6005AF3A1218970D
:012FC90022E5
:0D30CA00245265763A203439313620240036
:10252F00E529AB09AA0AA90B75F010A4F58285F06D
:10253F0083020BEBE493FF3395E0FEEF24D0FFEE25
:10254F0034FFFE7C00020C4CE52975F010A4AB099A
:10255F00250BF9E50A35F0FA900004020BEB900019
:10256F000D120E54785DE6FF18E68FF0A4FFE526F6
:10257F002FF582E435F0F583229006207478F078F9
:10258F0057E6241FF582E43405F583E022E53DC4C8
:10259F00F8540FC868FFE53CC454F04822785F90A8
:1025AF000521E0FCA3E0FDE6FA08E6FB22E527257E
:1025BF00262422F582E43405F583E022AB09AA0A2A
:1025CF00A90B2275F010A429F9EA35F0FA227860E8
:1025DF00900521E0FDE6FB229006207478F07F0144
:1025EF0022D20AC3ED9B785DF67859760122F582E7
:1025FF00E43405F58322D20A785DF67859229000EB
:10260F000D020E547B007A00792422900522E0FF00
:0F261F00E526D39F22E4F52B7875E614F52C22DF
:10125100E47880F61230A8C28575840F75E104E444
:10126100F5E275E344F58475B7B075840F758A832B
:10127100F597438901758D01758F01758E04F53CD4
:10128100F53D053DE53D7002053C640F453C70F2BE
:10129100438902E4F53CF53DAE3CAF3DE4FCFD7B0A
:1012A100507AC3F9F8D3120D1F400FE58920E40AE3
:1012B100053DE53D70E2053C80DE75970212301E6A
:1012C100E4FF12303D43EF04E4F53CF53D7D01AF11
:1012D1003D12000E053DE53D7002053CC39410E54D
:1012E1003C940040E8E4F520C20AC208C20EC20DD7
:1012F100C20C7880F608F67858F618F6785DF6F59F
:101301003CF53D7420253D1225FDE4F0053DE53D0C
:101311007002053CB400ECE53CB401E7E4F53CF5B2
:101321003D7420253DF582E43406F583E4F0053D66
:10133100E53D7002053C6440453C70E5E4F584E51B
:10134100EF20E10CE5EF5408D394004003D3800172
:10135100C392037D08E4FF122FF5E4785CF678551B
:10136100F61225CB7855E6FF122537FE785C26F676
:10137100EE600578550680E9EFD39400402A1225E6
:10138100CB12260D120BD2FF7455120C18120BD270
:1013910064556002D20C74AA120C18120BD264AA02
:1013A1006002D20CEF120C18E4F584E5EF5402D37D
:1013B100940040047F018002E4FF1226E98F3BE59F
:1013C1003B20E036C20974FF785FF608F608F6089C
:1013D100F67E007F107D007B007A007965120EAAEF
:1013E1007541FF75421B75437B7544007545107B44
:1013F100007A007965122D4B8002D2099030D17D9F
:1014010064122543AA06AB079030D0E493FF3395CD
:10141100E0FEEF24D0FFEE34FFFE7C037DE8120CEA
:101421004CEF2BFBEE3AFA9030D27D0A122543EFB6
:101431002BFFEE3AFEA3E493FD3395E0FCED24D0BF
:10144100FDEC34FFCD2F7864F6ED3E18F6E53B2038
:10145100E176E4F53CF53D12259CFE1225CB8F8209
:10146100F583120BEB6058E92FF9EA3E122566204D
:10147100E242E4F53AE53AC3787596503712259C75
:101481001225CB8F82F583120BEBFF7E00C006C0C5
:10149100077D0012259CFEE92FF9EA3EFA12260D7E
:1014A100785CE6853AF01225D5D007D006120EAA4F
:1014B100053A80C1053DE53D7002053C0214587FA7
:1014C100011216DFC20B8007E4FF1216DFD20BE414
:1014D100F53CF53D7A007B967D03AF3D122E3D052F
:1014E1003DE53D7002053CC39410E53C940040E4A9
:0114F10022D8
:05311A00785DE6FF22D4
:030023000224278D
:10242700C0E0C0F0C083C082C0D075D000C000C07B
:1024370001C002C003C004C005C006C00730993EF2
:10244700C2997858067958E77881667015F67858F2
:01245700F68E
:0D24580075220A75231300D523FCD522F64A
:04246500C285801C90
:0D24690075221475231300D523FCD522F62F
:102476007858E62420F582E43406F583E0F59920C1
:102486009803022514209A08200A05C298022510EE
:10249600C29A7857E60624201225FDE599F0C298DF
:1024A600E6FFB40112900520E0FE7003F6805FEEB1
:1024B60054072402785EF6EFB4020D785EE6B4099E
:1024C60007900521E02403F67857E6FFB40007E4F9
:1024D600B40103F68038EFC3785E9640317857E64C
:1024E60024FFFDE434FFFC7B017A057920122B2EB4
:0A24F60012258E6F6004760080143A
:0D25000075221475231300D523FCD522F697
:10250D0012002678577600D007D006D005D004D01B
:10251D0003D002D001D000D0D0D082D083D0F0D063
:02252D00E0329A
:102EDA008F348B358A368937E4F584EA494B601C8E
:102EEA00AB35AA36A937120BD2FFE534FD7C0012A6
:0C2EFA0030E4AB35AA36A937EF120C18F3
:0D2F060075381475391300D539FCD538F62F
:0E2F13008534997F011230793099FDC29922E0
:09305C00E4F5847881EFF6D285D9
:0D30650075341475351300D535FCD534F6DF
:07307200900620E0F5992211
:102F6200C9EFC9E96401701FEDC39B40277875E67C
:102F7200FFEB2FFFE433FEEDC39FEE6480F8748015
:102F82009850111225F022B90210ED6B700612262C
:0B2F920005760222C20AE47859F622FC
:102D9D00C9EFC9BAFF11BBFF0EED6B7002EC6A7083
:102DAD0038122605E9F622E96401701CC3ED9BEC8F
:102DBD009A40137875E62BFFE43AFEC3ED9FEC9E27
:102DCD0050041225F0228011B90214ED6B7002EC43
:102DDD006A7006122605760222C20AE47859F62296
:10002600900520E0FF54F8F525E4F584EF120E84E0
:10003600007309007A0A008110008A1100971200E5
:10004600A41900B41A00C82000D12801252901E707
:1000560033022237024C39025C4102674902715071
:1000660002AE6101B17002A698000002D31225DD2E
:100076007F0180171225AC7F01801DD20A78597640
:10008600030202D378621225DF7F02122F62020278
:10009600D378611225AE7F02122D9D0202D312255E
:1000A600DD7F01122F62200A030202D3800E122581
:1000B600AC7F01122D9D200A030202D31225E7020E
:1000C60002D0E4F58475EF100202D312074A7F18B6
:1000D6001207B47F05122EDA7855120732785F12AE
:1000E6000732786012073E786112073E786212077F
:1000F600627863120762786412077CE4F5267465F9
:0F0106002526F812077C0526E526C3941040EF46
:0D01150012078875331300D533FCD532F680
:1001220002019C900521E0FFC37855965073EF754C
:10013200F010A4250BF9E50A35F085092FF5308971
:100142003112074A7F0D122EDAAB2FAA30A93112D3
:10015200076E90000112070A90000212070A90002F
:100162000312071E90000412071EE4F526AB2FE5CA
:10017200312405F9E43530FA7E00E92526F9EE3A14
:0D018200FA12076E0526E526C3940840E03A
:0D018F0012078875331300D533FCD532F606
:10019C00C285D2AC0202D39006207478F0E4A3F0AE
:1001AC007F020202D01231067811120DC490062083
:1001BC00747CF07811E6A3F008E6A3F008E6A3F04F
:1001CC0008E6A3F07C007D057B017A067920122BD2
:1001DC002E900625EFF07F060202D0900521E0FF5D
:1001EC00B4010FA3E0FDA3E0785FCDF608EDF602B5
:1001FC0002A6EFB4020A900522E0785FF60202A68E
:10020C00900521E0B4030CA3E0FFA3E07861CFF6E6
:10021C0008EFF60202A6E4F526900521E0FFE5269C
:10022C00C39F5016742225261225C2FF74652526FD
:10023C00F8EFF60526E526B410DFE47874F6805A5C
:10024C001207A6900521E0FDE4FF122FF50202D360
:10025C00900521E024FF92020202D3900521E024B4
:10026C00FF92018062785DE66005752802800B20A4
:10027C000D0575280380037528019006207479F00C
:10028C00A3E528120797900622EFF07F0312305C4B
:10029C00E52864017031D20E8002D208788076F1A4
:1002AC0080257A007B327D017F00122E3D90062046
:1002BC007479F0900521E0900621120797900622A0
:1002CC00EFF07F0312305CE52564A0600302047C30
:1002DC00900520E064A1600302039DA3E0C3785560
:1002EC009640030203971225CBE0FF122537F52821
:1002FC00EF75F010A429F9EA12256430E22D90056F
:10030C0021E01200038F28900620747FF0A3E528CB
:10031C00F024021207C974222528F582E43406F56C
:10032C0083EFF0E5282403FF020479900521E0FF18
:10033C00120003C2ACE4F524D285E528D394064020
:10034C00221226137F7F1207B4AF28122EDAE4F59F
:10035C0026E526C3952850071206D2052680F205FD
:10036C00288018E52824781207BEE4F526E526C374
:0B037C00952850071206D2052680F2DB
:0D0387001207E375331300D533FCD532F6B1
:100394000204701225E7020479900520E064A2604B
:1003A4000302047C7855E6FFA3E0FEC39F400302EA
:1003B4000476A3E0FDC39F4003020476EE9D400350
:1003C400020476900521E0F526E4F52DF52E12269B
:1003D4001A5017AF26120003E526122531252EF5F3
:1003E4002EE4352DF52D052680E4C2ACE4F524D2A7
:1003F40085FB7A0079247F7F122EDAC3E52E948060
:10040400E52D940050028007E52D44801207BEAF0D
:100414002E122613122EDA900521E0F52612261A42
:10042400503DE4F5271225CB75F010E52612253A48
:10043400FFE527C39F5024E5261225D212260D7806
:100444005DE6FF18E68FF0A42527122580120BEB3A
:0F045400FF122613122EDA052780CA052680BE56
:0D0463001207E375331300D533FCD532F6D4
:10047000C285D2AC80061225E712305CE5256458AF
:10048000703BFA1207F27537017538067539217B12
:10049000017A0579211231118F28E52824789006F8
:1004A00020F0EF24011207C974212528F582E434D5
:1004B00006F583EFF0E5282402FF12305CE52564A1
:1004C000806009E525648860030205FC7859E6B47C
:1004D00001051207A68012E4F526E526C378759675
:1004E00050071207D7052680F1900520E05407F544
:1004F00028B4070A752701A3E0F528A38006E4F5D0
:1005000027900521E0F5291528E529C3785596405F
:10051000030205E612252FFFE528D39F40028F280E
:100520007859E6B40109785DE6F52CF52B800312C5
:100530002624785DA62B785DE6D3952C4003020532
:10054000DAE4F526E526C3952840030205CF1225F7
:100550005720E276900001120BEB64387036E528E4
:10056000D3940440061225BCFD80587857E6C39505
:1005700026FFE49400FE741E2FF58274053EF58379
:10058000E0FDE52975F010A4AB09250BF9E50A3566
:10059000F0FA802F12252FFF7857E6C39FFFE494CF
:1005A00000FE7C00EF2526FFEC3EFEEF2527FFEC4A
:1005B0003EFE741F2FF58274053EF583E0FDE529AC
:1005C0001225D212256DED120C2A0526020544AF24
:1005D0002912284C785D06020536785DA62BE525A4
:1005E000648870188010E529B4FF11900522E0F5A9
:1005F00020E525B488061225881207FEE52564A8A3
:1006000060030206D17859E6B401077A001207F2B6
:100610008012E4F526E526C378759650071207D7B1
:10062000052680F1900521E030E711547FFEA3E01C
:10063000FDEEF52DEDF52E752703800C900521E0DC
:10064000752D00F52E752702742025271225FDE053
:10065000FF74212527F582E43405F583E0F52A8F20
:1006600029E529D3952A5063E529C3785596505634
:1006700012252FF5287859E6B40109785DE6F52CA6
:10068000F52B8003122624785DA62B785DE6D395A2
:100690002C5029E4F526E526C39528501512255738
:1006A00020E20B1225BCFD12256DED120C2A052649
:1006B00080E4AF2912284C785D0680CF785DA62BA8
:1006C000E5282527F5270529020661122588120746
:0106D000FE2B
:1006D10022900521E075F010A4AB09250BF9E50A7C
:1006E10035F0FA90000D120E54785DE6FF18E68F92
:1006F100F0A42526F582E435F0F583120BEBFF7BA0
:10070100007A007924122EDA22AB2FAA30A93112F5
:100711000BEBFF7B007A007924122EDA22AB2FAA91
:1007210030A931120BEBFF7B007A007924122EDA0B
:1007310022E6FF7B007A007924122EDA22E6FF7B83
:10074100007A007924122EDA22C2ACE4F524D28593
:10075100FB7A0079247F7F122EDA7B007A007924DC
:1007610022E6FF7B007A007924122EDA22120BD2C4
:10077100FF7B007A007924122EDA22E6FF7B007AD1
:10078100007924122EDA227B007A007900AF24123C
:100791002EDA75320A22F07C007D027B017A06791D
:1007A10020122B2E227A007B327D01785DE6FF122A
:1007B1002E3D22122EDA7B007A00792422FF7B0063
:1007C1007A007924122EDA22FDE433FC7B017A06C9
:1007D1007920122B2E227A007B327D01AF26122E38
:1007E1003D227B007A007900AF24122EDA75320A9D
:1007F100227B327D01785DE6FF122E3D229006219B
:07080100F07F0212305C22BF
:10F000007880E664F1600302F60CE4F53FF54078A1
:04F0100081E6601F16
:0DF0140075450A75461300D546FCD545F636
:10F021000540E5407002053F64107004E53F642728
:10F0310070DCC2AF7584015398FC75FFDE75FFADBE
:10F04100E4F53BF53AE4F58420982EE4F53FF540EC
:0EF05100209822C3E5409488E53F94135017A1
:0DF05F0075450A75461300D546FCD545F6EB
:10F06C000540E54070DF053F80DBB2F880CF859925
:10F07C003AC298E53A641A600302F14CF53FF54048
:0EF08C00209822C3E5409488E53F9413501766
:0DF09A0075450A75461300D546FCD545F6B0
:10F0A7000540E54070DF053F80DB30989285993B4E
:10F0B700C298E4F53FF540209822C3E5409488E5DF
:05F0C7003F94135017F7
:0DF0CC0075450A75461300D546FCD545F67E
:10F0D9000540E54070DF053F80DB20980302F046DC
:10F0E90085993BC298E4F53FF540209822C3E54055
:08F0F9009488E53F94135017C1
:0DF1010075450A75461300D546FCD545F648
:10F10E000540E54070DF053F80DB20980302F046A6
:09F11E0085993BC298D285C29983
:0DF1270075451475461300D546FCD545F618
:06F134007599783099FD89
:0DF13A0075450A75461300D546FCD545F60F
:10F14700C28502F5FEE53A6450600302F1DCF53F43
:10F15700F540209822C3E5409488E53F9413501763
:0DF1670075450A75461300D546FCD545F6E2
:10F174000540E54070DF053F80DB20980302F04640
:09F1840085993BC298D285C2991D
:0DF18D0075451475461300D546FCD545F6B2
:08F19A007599793099FDC299C5
:0DF1A20075451475461300D546FCD545F69D
:08F1AF007599013099FDC29928
:0DF1B70075451475461300D546FCD545F688
:06F1C400E4F5993099FD0D
:0DF1CA0075450A75461300D546FCD545F67F
:0FF1D700C28502F5FEE53A6401703ED285C29909
:0DF1E60075451475461300D546FCD545F659
:08F1F3007599783099FDC2996D
:0DF1FB0075451475461300D546FCD545F644
:06F20800E4F5993099FDC8
:0DF20E0075450A75461300D546FCD545F63A
:10F21B00C28502F5FEE53A6402600302F2E2F53FB5
:10F22B00F540209822C3E5409488E53F941350178E
:0DF23B0075450A75461300D546FCD545F60D
:10F248000540E54070DF053F80DB20980302F0466B
:10F2580085993BC298E4F53CE53B13B392F8E53B4E
:10F2680025E0FEC3E49400EE94F0502AE53B7F00CD
:10F2780025E0FEC394E0501EE53B20E01FE4F58442
:10F2880043B701758F038E418F428F828E83F0536F
:10F29800B7F0F58F8003753CFFE4F584D285C299F9
:0DF2A80075451475461300D546FCD545F696
:08F2B5007599783099FDC299AA
:0DF2BD0075451475461300D546FCD545F681
:06F2CA00853C993099FD1E
:0DF2D00075450A75461300D546FCD545F678
:10F2DD00C28502F5FEE53A6403600302F42DF53FA5
:10F2ED00F540209822C3E5409488E53F94135017CC
:0DF2FD0075450A75461300D546FCD545F64B
:10F30A000540E54070DF053F80DB20980302F046A8
:10F31A0085993BC298E4F53FF540209822C3E54021
:08F32A009488E53F941350178D
:0DF3320075450A75461300D546FCD545F615
:10F33F000540E54070DF053F80DB20980302F04673
:10F34F0085993DC298E53B1392F8E53B25E0FEC356
:10F35F00E49400EE94F0400302F046E53B7D002577
:10F36F00E0FCC394E0400302F046E4F58443B701A8
:10F37F00758F01E53D75F020A42DFFE5F03CF541BB
:10F38F008F42E4F584F53EE53EC394205048E4F502
:10F39F003FF540209822C3E5409488E53F941350F1
:01F3AF001746
:0DF3B00075450A75461300D546FCD545F697
:10F3BD000540E54070DF053F80DB20980302F046F5
:10F3CD000542E542AE417002054114F5828E83E59A
:10F3DD0099F0C298053E80B1E4F58453B7F0F58FEE
:06F3ED00F584D285C299EF
:0DF3F30075451475461300D546FCD545F64A
:08F400007599783099FDC2995D
:0DF4080075451475461300D546FCD545F634
:06F41500E4F5993099FDB9
:0DF41B0075450A75461300D546FCD545F62B
:10F42800C28502F5FEE53A6404600302F4DDF53FA7
:10F43800F540209822C3E5409488E53F941350177F
:0DF4480075450A75461300D546FCD545F6FE
:10F455000540E54070DF053F80DB20980302F0465C
:10F4650085993BC298E53B25E0F543754400E4F5F5
:10F475003CF53FF5400544E544AE437002054314B1
:10F48500F5828E83E493253CF53C0540E54070020A
:0EF49500053F7004E53F640270DBD285C2992A
:0DF4A30075451475461300D546FCD545F699
:08F4B0007599783099FDC299AD
:0DF4B80075451475461300D546FCD545F684
:06F4C500853C993099FD21
:0DF4CB0075450A75461300D546FCD545F67B
:10F4D800C28502F5FEE53A6405600302F5F3F53FDF
:10F4E800F540209822C3E5409488E53F94135017CF
:0DF4F80075450A75461300D546FCD545F64E
:10F505000540E54070DF053F80DB20980302F046AB
:10F5150085993BC298E4F53FF540209822C3E54024
:08F525009488E53F9413501790
:0DF52D0075450A75461300D546FCD545F618
:10F53A000540E54070DF053F80DB20980302F04676
:09F54A0085993DC298D285C29951
:0DF5530075451475461300D546FCD545F6E8
:08F5600075997F3099FDC299F5
:0DF5680075451475461300D546FCD545F6D3
:10F575007599203099FDE53B25E0FCE53D75F020CA
:10F58500A42400FFE5F03CF5438F44E4F53CF53E4B
:02F59500C29919
:0DF5970075451475461300D546FCD545F6A4
:10F5A400854482854383E493F5993099FD0544E5C8
:10F5B40044AE437002054314F5828E83E493253CE4
:0BF5C400F53C053EE53EB420C8C299AE
:0DF5CF0075451475461300D546FCD545F66C
:06F5DC00853C993099FD09
:0DF5E20075450A75461300D546FCD545F663
:10F5EF00C285800BE53AB40606E4F58475EF10E5A5
:0DF5FF003A6407600302F0467880F6D2AF50
:01F60C0022DB
:102C8A007F0012307920090B7A007B327D017F00A8
:102C9A00122E3D300C0B7A007B1E7D017F00122E16
:102CAA003D300817300D147A007B327D01785DE6DD
:102CBA00FF122E3DC2081228F0D209200B0C300D4B
:102CCA0009788076F11228F0D20B300E08300D0503
:102CDA00C20E12F000200D121230FBE47B2C7A0196
:0B2CEA00F9F8C3120D355002D20D2284
:0B30F000121251122C8A122F9D80F842
:10231D00005EBCE2613FDD83C29C7E20A3FD1F41B8
:10232D009DC3217FFCA2401E5F01E3BD3E6082DCA8
:10233D00237D9FC1421CFEA0E1BF5D0380DE3C6298
:10234D00BEE0025CDF81633D7C22C09E1D43A1FF88
:10235D004618FAA427799BC584DA3866E5BB590778
:10236D00DB856739BAE406581947A5FB7826C49A68
:10237D00653BD987045AB8E6A7F91B45C6987A2458
:10238D00F8A6441A99C7257B3A6486D85B05E7B948
:10239D008CD2306EEDB3510F4E10F2AC2F7193CD38
:1023AD00114FADF3702ECC92D38D6F31B2EC0E5028
:1023BD00AFF1134DCE90722C6D33D18F0C52B0EE18
:1023CD00326C8ED0530DEFB1F0AE4C1291CF2D7308
:1023DD00CA947628ABF517490856B4EA6937D58BF8
:1023ED005709EBB536688AD495CB2977F4AA4816E8
:1023FD00E9B7550B88D6346A2B7597C94A14F6A8D8
:10240D00742AC896154BA9F7B6E80A54D7896B35C7
:0A241D00000000002B6096CBDDEEFE
:0330C600011D0ADF
:10262E00A810E6FF25E025E02464F582E43406F5E3
:10263E008322E53FAB09AA0AA90B75F010A4F58217
:10264E0085F083020BEBEF25E025E02462F582E4B2
:10265E003406F58322A8100808E624FF22EF25E0B1
:10266E0025E02461F582E43406F583221510A810C6
:10267E00EDF61510A810EFF62225E025E02463F5FF
:10268E0082E43406F58322EF2401FFE43EFEE43DAE
:10269E00FDE43CFC120DD09006602275F010A429CA
:1026AE00F9EA35F0FA90000D120E54785CE62278B5
:1026BE001DE675F064A4FFC3781FE69F18E695F03B
:1026CE0022A810E6FFC3941022120C942400FFE5FA
:0B26DE00F034E02215101510A81022A7
:102B2E001226E2ECF608EDF615101226E2120E4B06
:062B3E00E51024FCF51077
:102B4400F80808E4F6A810F608F6E5102407F9A832
:102B540010E6FE08E6FFC3099719E76480F8EE64FF
:102B640080985031E5102404F8120E328F828E833F
:102B7400120BEBA810080866FFE5102403F8EFF623
:102B8400E690231D93A8100808F6A8100806E61876
:0B2B940070B80680B5A8100808E6FF26
:072B9F00E5102409F51022E6
:0B30E400ED6F7815F6E690231D93FFBA
:0130EF0022BE
:102FF500EF7023F5847598D0F584759115F5847572
:10300500C90875CBFFED90241C93F5CA75C804E477
:08301500F584D2ACC2BCD2AFBD
:01301D002290
:102F21009006A1120DF5000000009006A5120DF506
:102F3100000000009006607464F0E47816F67816DC
:102F4100E6FFC39410501912266BE4F0122654E4E4
:102F5100F0EF122687E4F0EF122632E4F00680DE6D
:012F6100224D
:10301E00D2AFD2A9C2BBE4F584E589540F4401F5C1
:0F302E0089758E02758CAFE4F58AD28C022F2142
:022BA600151008
:102BA800A810E4F61226CF5067EF122632E0FFD3C2
:102BB80094004046E6122655E0703FEF30E00D12D3
:102BC8002630E0D3940140047D0180067D00A810E2
:102BD800E6FF12220D12262EE0B401057D00122216
:102BE8000D12262EE014F0EF122632E0600CE6FFFC
:102BF800122687E0FE122654EEF0A810E6FF1226F1
:102C080055E06006122654E014F0A81006022BAC1A
:032C180005102282
:03000B00022C1BA9
:102C1B00C0E0C0F0C083C082C0D0E8C0E0E9C0E033
:102C2B00EAC0E0EBC0E0ECC0E0EDC0E0EEC0E0EFEE
:102C3B00C0E0758CAF9006A1120D9F9006A11226D5
:102C4B0095E014F0E0700F9006A5120D9F9006A56D
:102C5B001226957464F0122BA6123094D0E0FFD09C
:102C6B00E0FED0E0FDD0E0FCD0E0FBD0E0FAD0E01D
:0F2C7B00F9D0E0F8D0D0D082D083D0F0D0E032C2
:10000E0012267A1226CF500808E6FE12266BEEF064
:05001E00051005102291
:102E3D001226E2EAF608EBF612267A1226CF503861
:102E4D00EF122632E07031E6FB122655E0702908AC
:102E5D00E625E004FFA810E6FA122632EFF0080886
:102E6D00E6FE08E6FF7C007D0A120C5EEA1226875C
:0F2E7D00EFF0EB122655E4F0E5102404F51022D7
:05220D0012267A1510F5
:10221200A81008E6FFC39410501912266BE0601351
:10222200A8100808E670047F0180027F00A8100849
:1022320008EFF6A810A68475840FA81008E6FF70B0
:102242000812266392F8022311EFB40108122663E2
:1022520092F9022311A81008E6FFB40208122663BD
:1022620092FA022311EFB4030812266392FB0223AF
:1022720011A81008E6FFB4040812266392FC022398
:1022820011EFB4050812266392FD022311A810086B
:10229200E6FFB4060812266392FE022311EFB4078A
:1022A2000812266392FF022311A81008E6FFB40861
:1022B2000712266392B08057EFB409071226639281
:1022C200B1804CA81008E6FFB40A0712266392B246
:1022D200803DEFB40B0712266392B38032A8100838
:1022E200E6FFB40C0712266392B48023EFB40D0705
:1022F20012266392B58018A81008E6FFB40E0712E2
:10230200266392B68009EFB40F0512266392B7A82E
:0423120010E6F58458
:07231600051005100510225F
:0A30FB00C2AF9006A1120D9FD2AFE4
:0131050022A7
:0A310600C2AF9006A5120D9FD2AFD4
:01311000229C
:10307900122680A810E67005781EF608F6300F08AB
:0B3089001226BD500375FFA5051022A4
:10303D00D20FE4781EF608F6EF781D6003F68002D5
:0F304D00760A75FF0775FFA5E4F58475EF042279
:1030A800C20FE4781EF608F6781D76FF75FFDE7508
:0330B800FFAD2247
:10309400781F06E618700106300F081226BD50038B
:0430A40075FFA522ED
:042FCA008E0C8F0DCD
:102FCE00E4F50EF50FC3E50F950DE50E950C5016B5
:102FDE007FE87E03122CF57F01123079050FE50F85
:062FEE0070E3050E80DF18
:012FF40022BA
:042CF5008E4D8F4E23
:102CF900D3E54E94FAE54D9400500EEFD39400407D
:102D0900407E1600DEFD1F80F2854D4F854E50D363
:102D1900E55094FAE54F940040157FFA7E00122C95
:102D2900F574062550F55074FF354FF54F80E0D303
:102D3900E54E9400E54D94004007AF50AE4F122C7C
:012D4900F594
:012D4A002266
:082DED008B468A4789488D4995
:102DF5007F01123079AB4AAA4BA94C1226D7FE8522
:102E0500464D85474E85484FE4FDEDC39549501B1A
:102E1500EF2DF582E43EF583E493AB4DAA4EA94F21
:102E25008D82758300120C2A0D80DFAB4AAA4BA94F
:082E35004CE48549F0020CBFDA
:082AA8008B408A4189428D43F5
:102AB0007880E664F170761230A8C2AFE4F5844302
:102AC000B701758F01AB44AA45A9461226D77816DF
:102AD000F608EFF6AB40AA41A942781A120E4BE471
:102AE0007818F67818E6C395435029781AE475F0FB
:102AF00001120E3B120BD27819F6E6FF7816080683
:102B0000E618CCE6CC70010614F5828C83EFF078E1
:102B1000180680CFE4F58F53B7F0AB44AA45A94619
:0D2B20008543F0120CBFD2AFE4FF12303D30
:012B2D002285
:102E8C007880E664F17046C2AF1230A8E4F5844352
:102E9C00B701758F03781776E008F67816F6781771
:102EAC00E6FE08E6F5828E83E4F07F011230797835
:102EBC0018E426F618740236F61806E6C394084091
:0D2ECC00DDE4F58F53B7F0D2AFFF12303DBB
:012ED90022D6
:1028F000122E8CE4F53EF53FF54475450075463ED5
:10290000FB7A00795F7D16122AA812296CF53BE547
:102910003BC3787596504EE4F53AE53A122642608C
:1029200040E53A1226A9853BF0A429F9EA35F0FAE8
:10293000EBC0E0EAC0E0E9C0E0AB09AA0AA90B7568
:10294000F010E53A12264BFD7544007545007546BA
:102950003ED0E0F9D0E0FAD0E0FB122AA8053A8098
:0B296000B9053B80AA12296C7880F6B4
:10296B0022753C12753D3475440075450075463E25
:0D297B007B007A00793C7D02122AA8E4223C
:0226E9008F3E22
:1026EB00E4F544F545F541F54A754B00754C44FB53
:1026FB007A00795F7D16122DED1227837004E54267
:10270B0064127003434101E4F540E540C3787596CC
:10271B005055E4F53F1226406048E53E6033E53FF7
:10272B001226A98540F0A429F9EA35F0FAEBC0E0AE
:10273B00EAC0E0E9C0E0122640FD754A00754B0087
:10274B00754C44D0E0F9D0E0FAD0E0FB122DED80CF
:10275B000C1226402545F545E43544F544053F026A
:10276B00272005400227151227837004E5426412C7
:07277B007003434102AF416E
:1027820022754A00754B00754C447B007A007942F1
:0A2792007D02122DEDE543643422B0
:10080800020BBDE86480F8E933E83360110460F056
:10081800ED33EC337009E8FCE9FDEAFEEBFF220456
:1008280060DED3EB9FEA9EE99DE8C2E78CF0C2F751
:1008380095F0400CE8CCF8E9CDF9EACEFAEBCFFB1D
:10084800120B8885D0F05804700320D5B3E80470E3
:10085800075002B2D5020BC792D5EC0460F7E4CC7E
:10086800C0E0C398F8603B94186008400DD0E0FBE6
:10087800020B9FE4FBFAC9FC8028E830E406E4C9CF
:10088800FBE4CAFCE830E305E4C9CACBFCE854073A
:100898006010F8C3E913F9EA13FAEB13FBEC13FC45
:1008A800D8F130F52FC3E49CFCEF9BFFEE9AFEEDE8
:1008B80099FDD0E0FBEF4E4D4C701222DB03020B8A
:1008C800C4EC2CFCEF33FFEE33FEED33FDED30E7E7
:1008D800EB020B9FEF2BFFEE3AFEED39FDD0E0FB6C
:1008E80050130BBB0003020BC7ED13FDEE13FEEF15
:0808F80013FFEC13FC020B9F3F
:10090000EC4D6011E8497017ED33EC3304600DE4F1
:10091000FCFFFEFD22E933E8330470F8020BBD1240
:100920000B8858046009E4CC248150062850090241
:100930000BC7284003020BC4C0E0EB4A7044B980E7
:1009400006D0E0FB020BB3EF4E701CBD8008EBFF3E
:10095000EAFEE9FD80EBE98DF0A4FEE5F00209E98D
:10096000E9CDF9EAFEEBFFEF89F0A4FCE5F0CE89D2
:10097000F0A42EFFE435F0CD89F0A42DFEE435F08F
:100980008067EF4E7005BD80D780C3EF8BF0A4ACBD
:10099000F0EE8BF0A42CFCE435F0F8EF8AF0A42CF8
:1009A000E5F038FCE433CB8DF0A42CFCE5F03BF80B
:1009B000EE8AF0A42CFCE5F038F8E433CF89F0A4FB
:1009C0002CFCE5F038CF3400CE89F0A42FFFE5F001
:1009D0003EFEE433C98DF0A42EFEE5F039CD8AF059
:1009E000A42FFFE5F03EFEE43DFD33D0E0FB5007D1
:1009F0000BBB000F020BC7EC2CFCEF33FFEE33FEFA
:060A0000ED33FD020B9F27
:100A0600020BC7EC5D046005E859047003020BBDD8
:100A1600120B88580460F6EC4860F2EC7004FDFE98
:100A2600FF22C860DB2481C85009C39860025006C3
:100A3600020BC49850CAF582E9294B4A7005AB826D
:100A4600020BB375F0007C1A7880C3EF9BEE9AED2B
:100A560099400DC3EF9BFFEE9AFEED99FDE842F03B
:100A6600DC23ACF0D0E0FFD0E0FED0E0FDAB82208E
:100A7600E7101BEB60BAEC2CFCEF33FFEE33FEED18
:100A860033FD020B9FE803F830E705C0F075F00070
:100A9600EF2FFFEE33FEED33FD40B830E7C280AAFC
:100AA60074F8CC6480CCC86480C8F582046043C303
:100AB600EB9FF5F0EA9E42F0E99D42F0E89C45F096
:100AC60060305018E5825FFFE582F42B5582FB50BB
:100AD600210ABA001D09B90019088016E5825BFBD8
:100AE600E582F42F5582FF50090EBE00050DBD00AC
:100AF600010CC3EB9FF5F0EA9E42F0E99D42F0E857
:0D0B06009C45F06007CC4820E701B3EC22CD
:100B130075F020800E75F010800575F0087D007E5D
:100B2300007F003392D530D503120D11EC33401002
:100B3300EF33FFEE33FEED33FDEC33FCD5F0ED2266
:0E0B4300E5F0247EA2D513CC92E7CDCEFF22A2
:100B5100EDD2E7CD33EC3392D524814006E4FFFE9C
:100B6100FDFC22FCE4CFCECDCC24E0501174FF80FB
:100B7100EDC3CC13CCCD13CDCE13CECF13CF047098
:070B8100F030D5DE020D117A
:0D30D700ED33EC3360065004EC6480FC2205
:10279C008F508E4F8D4E8C4D74FFFFFEFDFCAB5059
:1027AC00AA4FA94EA84DC3120D35602C7F807E9682
:1027BC007D187C4BAB50AA4FA94EA84D120AA660AF
:1027CC000250157F807E967D187CCBAB50AA4FA90A
:1027DC004EA84D120AA65009AF50AE4FAD4EAC4D9F
:1027EC0022AF50AE4FAD4EAC4D120B518F548E5399
:1027FC008D528C51EC120B13C8ECC8C9EDC9CAEE42
:10280C00CACBEFCBAF50AE4FAD4EAC4D12080BE474
:10281C00FBFAF9F8120AA6601A401874FF2554F551
:10282C0054E55334FFF553E55234FFF552E551347A
:10283C00FFF551AF54AE53AD52AC51EC120B132209
:100B8800E9D2E7C933E833F892D5EDD2E7CD33ECB3
:070B980033FC5002B2D5222C
:100B9F00EC30E7100FBF000C0EBE00080DBD0004B7
:100BAF000BEB6014A2D5EB13FCED92E7FD2274FF63
:100BBF00FCFDFEFF22E480F8A2D574FF13FC7D80BC
:030BCF00E480EFD0
:03000000022A1CB5
:0C2A1C00787FE4F6D8FD758181022A6302
:100BD200BB010689828A83E0225002E722BBFE0221
:090BE200E32289828A83E4932254
:100BEB00BB010CE58229F582E5833AF583E02250BF
:100BFB0006E92582F8E622BBFE06E92582F8E22209
:0D0C0B00E58229F582E5833AF583E4932222
:100C1800BB010689828A83F0225002F722BBFE01BB
:020C2800F322B5
:100C2A00F8BB010DE58229F582E5833AF583E8F000
:100C3A00225006E92582C8F622BBFE05E92582C8AC
:020C4A00F22294
:100C4C00EF8DF0A4A8F0CF8CF0A428CE8DF0A42EBC
:020C5C00FE2276
:100C5E00C2D5EC30E709B2D5E4C39DFDE49CFCEEB1
:100C6E0030E715B2D5E4C39FFFE49EFE120ED6C345
:100C7E00E49DFDE49CFC8003120ED630D507C3E440
:060C8E009FFFE49EFE2220
:100C9400BB010A89828A83E0F5F0A3E0225006872B
:100CA400F009E71922BBFE07E3F5F009E3192289ED
:0B0CB400828A83E493F5F07401932220
:100CBF00BB010789828A83020F2B500B09C5F027CE
:100CCF00F7C5F01937F722BBFE0D09F8E325F0F34E
:100CDF00C5F019E338F322F889828A8374019325CA
:080CEF00F0C5F0F8E49338228F
:0D0CF700EF2BFFEE3AFEED39FDEC38FC224C
:0D0D0400EF4BFFEE4AFEED49FDEC48FC22EE
:0E0D1100C3E49FFFE49EFEE49DFDE49CFC22F3
:100D1F00EB9FF5F0EA9E42F0E99D42F0EC6480C84B
:060D2F0064809845F022EB
:100D3500EB9FF5F0EA9E42F0E99D42F0E89C45F014
:010D4500228B
:100D4600E8600FEFC333FFEE33FEED33FDEC33FC0B
:030D5600D8F122AF
:100D5900BB010789828A83020D9F5005E9F8020DBC
:100D690093BBFE05E9F8020F4189828A83020F4D80
:100D7900BB010789828A83020DD05005E9F8020D6B
:0A0D8900C4BBFE05E9F8020F5D226D
:0C0D9300E6FC08E6FD08E6FE08E6FF228C
:0C0D9F00E0FCA3E0FDA3E0FEA3E0FF22C7
:0D0DAB00E6FB08E6F908E6FA08E6CBF822B8
:0C0DB800E0F8A3E0F9A3E0FAA3E0FB22BE
:0C0DC400ECF608EDF608EEF608EFF6225B
:0C0DD000ECF0A3EDF0A3EEF0A3EFF02296
:100DDC00D083D082E493F608740193F608740293DE
:090DEC00F608740393F674047315
:100DF500A8828583F0D083D082120E0C120E0C12BD
:100E05000E0C120E0CE473E493A3C583C5F0C583E1
:100E1500C8C582C8F0A3C583C5F0C583C8C582C847
:010E250022AA
:0C0E2600A42582F582E5F03583F58322D7
:090E3200E6FB08E6FA08E6F922E5
:100E3B00FAE6FB0808E6F925F0F618E6CA3AF622B8
:090E4B00EBF608EAF608E9F622CC
:100E5400BB010DE58229F582E5833AF583020F692A
:100E64005007E92582F8020E32BBFE07E92582F815
:100E7400020F72E58229F582E5833AF583020F7B3E
:100E8400D083D082F8E4937012740193700DA3A3FD
:100E940093F8740193F5828883E473740293686011
:060EA400EFA3A3A380DF11
:102D4B008B3E8A3F8940E4F546F547E5451545AE90
:102D5B0044700215444E6033AB41AA42A943120B97
:102D6B00D2FFAB3EAA3FA9400547E547AC467002F0
:102D7B00054614F5828C83EF120C2AEF60CD74019B
:102D8B002543F543E43542F54280C0AB3EAA3FA94B
:022D9B004022D4
:100EAA00EF4E6012EF60010EEDBB010B89828A835F
:100EBA00F0A3DFFCDEFA2289F05007F709DFFCA96C
:0C0ECA00F022BBFEFCF309DFFCA9F022C3
:102A28000230F0E493A3F8E493A34003F68001F2A4
:102A380008DFF48029E493A3F85407240CC8C333AF
:102A4800C4540F4420C8834004F456800146F6DF7E
:102A5800E4800B01020408102040809030BBE47E23
:102A6800019360BCA3FF543F30E509541FFEE49373
:102A7800A360010ECF54C025E060A840B8E493A33A
:102A8800FAE493A3F8E493A3C8C582C8CAC583CA65
:102A9800F0A3C8C582C8CAC583CADFE9DEE780BE1D
:0130C9000006
:100ED600BC000BBE0029EF8DF084FFADF022E4CC00
:100EE600F875F008EF2FFFEE33FEEC33FCEE9DECC9
:100EF600984005FCEE9DFE0FD5F0E9E4CEFD22ED0F
:100F0600F8F5F0EE8420D21CFEADF075F008EF2F58
:100F1600FFED33FD4007985006D5F0F222C398FD49
:050F26000FD5F0EA22E6
:100F2B00C5F0F8A3E028F0C5F0F8E5821582700251
:060F3B001583E038F022EE
:0C0F4100E2FC08E2FD08E2FE08E2FF22EC
:100F4D00E493FC740193FD740293FE740393FF22EA
:0C0F5D00ECF208EDF208EEF208EFF222D0
:090F6900E0FBA3E0FAA3E0F92289
:090F7200E2FB08E2FA08E2F922B0
:0C0F7B00E493FB740193FA740293F922D2
:00000001FF
